:020000020000FC
:10000000E3E0EEBFE0E0EDBF239A539A559A229ABF
:10001000549A219A579A3B9A2ED1EF93FF93E8EE88
:10002000F3E0EF93FF93ECECF7E03197F1F7FF91FA
:10003000EF91319711F000C0F4CFEF91FF915EE1A5
:100040005F9A439AE52F5C9A2B9AEF93FF93E4E033
:10005000F0E0EF93FF93ECECF7E03197F1F7FF91CD
:10006000EF91319711F000C0F4CFEF91FF912B98F1
:10007000EF93FF93E0E1F0E0EF93FF93ECECF7E018
:100080003197F1F7FF91EF91319711F000C0F4CF64
:10009000EF91FF91EA9509F0D6CF2B985C985F9885
:1000A0004398E52F299A2B9AEF93FF93E4E0F0E031
:1000B000EF93FF93ECECF7E03197F1F7FF91EF91BD
:1000C000319711F000C0F4CFEF91FF912B98EF938F
:1000D000FF93E0E1F0E0EF93FF93ECECF7E0319772
:1000E000F1F7FF91EF91319711F000C0F4CFEF914C
:1000F000FF91EA9509F0D6CF29982B985F9A439AF9
:10010000E52F299A5B9AEF93FF93E4E0F0E0EF93F9
:10011000FF93ECECF7E03197F1F7FF91EF91319716
:1001200011F000C0F4CFEF91FF915B98EF93FF9334
:10013000E0E1F0E0EF93FF93ECECF7E03197F1F7BB
:10014000FF91EF91319711F000C0F4CFEF91FF9143
:10015000EA9509F0D6CF29985B985F984398E52FE8
:100160002A9A5B9AEF93FF93E4E0F0E0EF93FF931A
:10017000ECECF7E03197F1F7FF91EF91319711F047
:1001800000C0F4CFEF91FF915B98EF93FF93E0E114
:10019000F0E0EF93FF93ECECF7E03197F1F7FF918C
:1001A000EF91319711F000C0F4CFEF91FF91EA95F4
:1001B00009F0D6CF2A985B985F9A439AE52F2A9A3E
:1001C0005D9AEF93FF93E4E0F0E0EF93FF93ECECA4
:1001D000F7E03197F1F7FF91EF91319711F000C0FF
:1001E000F4CFEF91FF915D98EF93FF93E0E1F0E0A2
:1001F000EF93FF93ECECF7E03197F1F7FF91EF917C
:10020000319711F000C0F4CFEF91FF91EA9509F01A
:10021000D6CF2A985D985F984398E52F5C9A5D9AAF
:10022000EF93FF93E4E0F0E0EF93FF93ECECF7E063
:100230003197F1F7FF91EF91319711F000C0F4CFB2
:10024000EF91FF915D98EF93FF93E0E1F0E0EF9382
:10025000FF93ECECF7E03197F1F7FF91EF913197D5
:1002600011F000C0F4CFEF91FF91EA9509F0D6CFDD
:100270005C985D98E5CE5F9AEF93FF93E8EEF3E02C
:10028000EF93FF93ECECF7E03197F1F7FF91EF91EB
:10029000319711F000C0F4CFEF91FF91439AEF93A3
:1002A000FF93E8EEF3E0EF93FF93ECECF7E0319788
:1002B000F1F7FF91EF91319711F000C0F4CFEF917A
:1002C000FF914398EF93FF93E8EEF3E0EF93FF93F2
:1002D000ECECF7E03197F1F7FF91EF91319711F0E6
:0C02E00000C0F4CFEF91FF915F980895EB
:00000001FF
